:020000040000FA
:100000000C2BC101C001C201C110BD010030B20002
:100010000530B3007C22A9220030B2008430B30046
:100020007C220430B2008030B3007C222030B20049
:10003000B3017C220F30B200F030B3007C220B30D1
:10004000B2000F30B3007C220D30B2000F30B3008D
:100050007C220930B2005030B3007C220730B2005D
:10006000D630B3007C224D222730B2000130B300DD
:100070007C220530B2000230B3007C220030B20096
:100080008C30B3007C2207306B22BB000730B200FB
:10009000B3017C223B08B3007C2A2A306B22BA00D1
:1000A0003A1F0800BA1E0800F122263084000430EE
:1000B000AF002930B2008422672A06306B22BB00D1
:1000C0003B1F68280C306B22BB003B18B22808008D
:1000D0003B1D72280A306B22BB003B182229BB183B
:1000E0004D2808003B1E7A280E306B22BB003B1ABD
:1000F000442A0800BB1C080008306B22BB003B1FD1
:100100009A280530B2000030B3007C220430B200DF
:100110008030B3007C222030B200B3017C224D221B
:100120002730B2000130B3007C220530B20002302B
:10013000B3007C2A3B1EA6280930B200C030B300B1
:100140007C220530B2000330B3007C2ABB1F0800BC
:100150000930B2005030B3007C220530B2000230CA
:10016000B3007C2A26306B22B900391F192944308C
:1001700084000830AF002530B200712254224D2295
:100180002030A42244086039031D10294508063A8E
:10019000031DCC284D2112294508013A031DD22800
:1001A000342112294508083A031DDC282130B20009
:1001B0003D08B3007C2212294508003A031DE228BD
:1001C000C521122945080A3A031DEB282130B20047
:1001D000B3017C2212294508053A031DFC28203072
:1001E000B2004030B3007C220430B20046088038B0
:1001F000BC00B3007C2212294508093A031D0229DC
:10020000FB2112294508033A031D0829152212294A
:1002100045080B3A031D10294608003A0319122914
:1002200020309F222330B2000530B3007C224210E0
:100230000800C11C1D29C1104D222730B200013019
:10024000B3007C2A22306B22BA003A1F3329BA1E2F
:1002500033294D22C11C2E292C22562A2730B200C8
:100260000130B3007C2A080044080339023A031D18
:1002700008004808C30043080F39C300003A031DB3
:1002800045292030A422401008004308013A031DEC
:1002900008002830A422C0100800C1144708B60086
:1002A0003608013A031D5829B7011230B800B929A0
:1002B0003608023A031D61291230B7006830B800D1
:1002C000B9293608213A031D6A292430B7002D3098
:1002D000B800B9293608223A031D73293430B70013
:1002E0006830B800B9293608043A031D7C291B3050
:1002F000B7002430B800B9293608033A031DB729DE
:1003000046088000003A031D8A296830B7006C3027
:10031000B800B9294608013A031D93296C30B7008B
:100320007A30B800B9294608023A031D9C297A3070
:10033000B700A030B800B9294608033A031DA52923
:10034000A030B700AE30B800B9294608043A031D02
:10035000AE29AE30B700B430B800B9294608053A26
:10036000031DB729B430B700BA30B800B929B701B6
:10037000B8014B08031DC429370838024A02031884
:10038000C4294A083707B8002C2A44080339C30097
:10039000003A031DD1292130B2000130B3007C2284
:1003A000E4294308013A031DDA292108B200B30108
:1003B0007C22E4294308023A031DE4294808C300CB
:1003C00043080F39C300E8212130B200B3017C2A71
:1003D000C30AB0010314B00DC30BEB294008B005EC
:1003E0000319F7292130B2000130B3007C2A2130F3
:1003F000B200B3017C2A4608BD00003A0319112A55
:10040000C201C00152222830B2001130B3007C2258
:10041000F122263084000430AF002930B20084225B
:10042000672A2830B200B3017C2A44080339023A13
:10043000031D080048080F39C800003A031D242A8C
:1004400020309F22401408004808013A031D08008C
:1004500028309F22C01408000830AF003708380247
:10046000083C031C382A3708380203190800AF007B
:100470002130C03805118F22370822238F22B70A76
:10048000AF0B3C2A05150800C11C0800C1104D2205
:100490002730B2000130B3007C2A2330B20008308C
:1004A000B3007C2A2B304E2A27304E2A2330B2004C
:1004B000013042180438B3007C220130C206080023
:1004C0002B30B2000330C2180438B3007C2A6022FB
:1004D0000230C206080005118F2203018F22051584
:1004E0000800051132088F2232088F228000840A0A
:1004F000AF0B742A051508000511320880388F22C9
:1005000033088F220515080005113208C0388F22E4
:1005100000088F22840AAF0B882A05150800B40052
:100520000830B500B40D05120318051685163410F1
:10053000851934148512B50B922A34080800B200CC
:100540006B228017B3007C2AB2006B228013B300A9
:100550007C2AFA30B100AF22B10BAB2A0800B001FF
:10056000B00BB02A080003306B220830A000031043
:1005700005180314A50D85168512A00BB72A3F3068
:10058000A5050800A601A701A801A90109302505B4
:10059000031DCC2A2615D02A251CA614A51D261419
:1005A000123025050319E32A2308A51CA707251ED9
:1005B000A70224302505031908002308A51EA80258
:1005C000251DA80708000230A106A11C0800243040
:1005D0002505031908000130A51EA907251DA9023C
:1005E0000800B322250936390319A201240825047D
:1005F000363A3639031DFE2AA201022B0C302202A4
:10060000031CA20A03302202031C0030A3000230A4
:10061000A3072508A400C22AFF2383169000873071
:1006200081008B010B308500831207309900043064
:1006300085000130A3003F30A400A20101208518ED
:100640005D201F2BAE0003308A002E088207123473
:100650000134103401340034003400340834DA3406
:100660000834813403340134003401340234033457
:1006700001340934023422340034013401340434A6
:100680008034323409340434013400340134033406
:100690000134023405340934213400340134003487
:1006A00001342234343400340734053481340334C3
:1006B0000434003432340534013409340234A134B2
:1006C000013409340134A1340034053409341934B7
:1006D000013429340334153400342534013495347D
:1006E0000334753401348134023495340134753463
:1006F000053481340134053401340934303409348B
:100700003134093438341534813425347F34753428
:1007100008349534033481340634C034C03404348E
:100720000334093404340E3403344A3400344A3474
:100730000034313400344F340034443400344D3408
:100740000034263403344A3400344F3400345934EE
:100750000034503400344134003444340034203404
:1007600000345734003448340034453400344534C0
:1007700000344C340034203400344D3400344F34D1
:1007800000345534003453340034453400340E34CE
:1007900003344A340034573400344D340034303498
:1007A00000343034003431340034063403344234FD
:1007B000003461340034063403343134003470348E
:0207C000003403
:02400E00C43FAD
:00000001FF
